:10000000AAC00000C4C00000C2C00000C0C0000000
:10001000BEC00000BCC00000BAC00000B8C00000F4
:10002000B6C00000B4C000000C94BE09B0C000000F
:10003000AEC00000ACC00000AAC00000A8C0000014
:10004000A6C00000A4C00000A2C00000A0C0000024
:100050009EC000006DC100009AC0000099C0000061
:1000600096C0000025C3000092C0000090C00000B0
:100070008EC000008CC000008AC0000088C0000054
:1000800086C0000084C0000082C0000080C0000064
:100090007EC000007CC000007AC0000078C0000074
:1000A00076C0000074C0000072C000000600FF09A6
:1000B00001A1010902150025FF75089508810209B3
:1000C00003150025FF750895089102C01201100163
:1000D000000000085423222200020102000109024C
:1000E0002200010100C0FA09040000010300000021
:1000F00009211101000122200007058103080001E8
:10010000040309042E0342006900720064004200E7
:100110007200610069006E002000540065006300F9
:1001200068006E006F006C006F006700690065007A
:10013000730000002003480075006D006D00690029
:100140006E006700620069007200640020004400D5
:1001500075006F00000011241FBECFEFDAE0DEBF94
:10016000CDBF11E0A0E0B1E0EEEAFCE102C00590F5
:100170000D92A031B107D9F713E0A0E1B1E001C0C1
:100180001D92A136B107E1F730D30C94550E38CF4C
:100190001F920F920FB60F9211242F933F938F93BC
:1001A0009F93AF93BF93EF93FF9380912701882391
:1001B000F9F490912801953118F09093250102C02F
:1001C0001092250180912901882311F49F5F01C0BD
:1001D000915090932801809128018E3F20F081E07A
:1001E000809329010AC0833040F41092290105C090
:1001F000813019F48FEF8093250120E030E0F90180
:10020000E05FFE4FD901A55EBE4F8C9180832F5FCA
:100210003F4F2B30310599F780911001882311F061
:10022000769A04C076988FEF809310018091110127
:10023000882311F05C9A04C05C988FEF80931101C1
:1002400080911201882311F05E9A04C05E988FEFAE
:100250008093120180911301882311F0469A04C003
:1002600046988FEF8093130180911401882311F039
:100270005F9A04C05F988FEF8093140180911501FD
:10028000882311F02F9A04C02F988FEF80931501C7
:1002900080911601882311F0589A04C058988FEF66
:1002A0008093160180911701882311F0599A04C098
:1002B00059988FEF8093170180911801882311F0CE
:1002C000729A04C072988FEF80931801809119017F
:1002D000882311F08F9A04C08F988FEF80931901B3
:1002E00080911A01882331F0479A80912601E0E13C
:1002F000F1E005C047988FEF80931A01F6CF908107
:10030000981708F4892F319691E0EB31F907B9F786
:100310008093260187BDFF91EF91BF91AF919F918F
:100320008F913F912F910F900FBE0F901F901895B6
:100330001F920F920FB60F9211248F939F93EF93FA
:10034000FF93909126019F3F09F467C080911001AF
:10035000891721F476988FEF809310018091110115
:10036000891721F45C988FEF80931101809112011D
:10037000891721F45E988FEF809312018091130109
:10038000891721F446988FEF80931301809114010F
:10039000891721F45F988FEF8093140180911501E4
:1003A000891721F42F988FEF809315018091160102
:1003B000891721F458988FEF8093160180911701C7
:1003C000891721F459988FEF8093170180911801B4
:1003D000891721F472988FEF809318018091190189
:1003E000891721F48F988FEF8093190180911A015A
:1003F000891721F447988FEF80931A01E0E1F1E02B
:100400008FEF9081981708F4892F319691E0EB31A6
:10041000F907B9F78093260187BDFF91EF919F916E
:100420008F910F900FBE0F901F90189514BC84E011
:1004300085BD83E080936E00279A87B1806C87B971
:100440008AB1836D8AB98DB184648DB9879A089514
:1004500080931B0160931C0140931D0108958093BC
:100460001E0160931F01409320010895813321F400
:10047000CB01BA01A901F3CFCB01BA01A901E8CFA1
:100480008093210108958093220108958093230190
:100490000895809324010895813361F0823318F424
:1004A000803371F405C0823339F0833349F406C0D8
:1004B000CB01E6CFCB01E7CFCB01E8CFCB01E9CF32
:1004C000089580E090E060E070E040E050E0C0DF40
:1004D00080E090E060E070E040E050E0C0DF80E06D
:1004E00090E0CEDF80E090E0CEDF80E090E0CEDFF5
:1004F00080E090E0CECF80E680937C0084E880931B
:100500007A0010927B0083E780937E0008958093A9
:100510007C0080917A00806480937A0080917A00D8
:1005200086FDFCCF80917A00806180937A00809173
:10053000790090E0089584B1866184B985E58CBD29
:100540002C9A08952C989AE69A95F1F78EBD0DB4E1
:1005500007FEFDCF85ED8A95F1F72C9A08958EEF71
:10056000F1CFEF92FF920F931F93082FF62EE42EF8
:10057000982F9C5F862F880F890FE4DF88EC90E02E
:100580000197F1F78E2DDEDF10E0000F111FEAE278
:10059000F1E0DF01A00FB11FFC92FD01E1821F918C
:1005A0000F91FF90EF9008958FEFCCCF0F931F9393
:1005B000182F062FC7DF88EC90E00197F1F7802F06
:1005C000C1DFEEE2F1E0E10FF11D00831F910F9119
:1005D0000895262F30E0803339F43093890020933A
:1005E000880060933201089530938B0020938A0035
:1005F0006093330108951092890010928800109240
:100600008B0010928A0010923201109233010895EB
:1006100081EA8093800089E08093810084B18066C4
:1006200084B9E9CF82E08093C80088E98093C9004B
:1006300086E08093CA00109252031092530380E127
:100640008093CC000895982F8091C80085FFFCCF3F
:100650009093CE000895909152038091530320E02F
:10066000981321E0822F08951F9380915303E2E5B0
:10067000F2E0E80FF11D1081809153038F5F8093AA
:100680005303812FE0DF812F1F9108959091520332
:100690009F5F809153032091CE00981741F0E09125
:1006A0005203F0E0EE5AFD4F2083909352030895D9
:1006B0001F920F920FB60F9211242F933F934F93D7
:1006C0005F936F937F938F939F93AF93BF93EF93BA
:1006D000FF93DCDFFF91EF91BF91AF919F918F91DD
:1006E0007F916F915F914F913F912F910F900FBE2E
:1006F0000F901F90189508951092270130DFE1DECA
:1007000053DF79CF80910E0190910F01009729F06E
:10071000019790930F0180930E0108950F931F93FB
:10072000A801ECE3F2E060933C026093470200937F
:100730003D02528300934802509349023396CF0101
:10074000B9010E94450E1F910F9108950F931F93B9
:10075000CF93DF93FB01C901E801209147022111EA
:1007600020832AE432E04091480250914902B901C5
:100770000E94450E80914802909149029983888396
:1007800080E0DF91CF911F910F91089580E091E07B
:100790000C94F30C80E091E00E94D20CE2EEF0E0C9
:1007A000808184608083089584B7877F84BF88E1D7
:1007B0000FB6F89480936000109260000FBE80E046
:1007C00090E020E80FB6F8942093610080936100D8
:1007D0000FBE209A289A559A5D9A3F9A47988BDEC9
:1007E00025DE16DFA8DEADD51DCF2F923F924F92AA
:1007F0005F926F927F928F929F92AF92BF92CF92B1
:10080000DF92EF92FF920F931F93DF93CF93CDB7B9
:10081000DEB72E970FB6F894DEBF0FBECDBFC4DF94
:10082000789466247724AA24BB24650150E2E52E3F
:1008300051EAF52E57E0052F112D99248824839431
:1008400040E4442E4FE1542E32E0232E312C2C0E66
:100850003D1ECE0104969C878B87FE013596FE8750
:10086000ED87CE0106969A8789870AC0AA24BB2401
:10087000650120E4E22E2BE4F22E2CE4022F112D50
:1008800080E091E0C0D7AAD7AE14BF04C006D1065D
:1008900089F4D601C5010596A11DB11D8A159B05D8
:1008A000AC05BD0588F05BDE0CDE7EDEA4DE1092BA
:1008B000270105C0AE14BF04C006D10628F4089471
:1008C000A11CB11CC11CD11CC6DE882309F488C13F
:1008D000CBDE8983823509F406C1833580F48C34FC
:1008E00009F447C08D3420F4873409F0C2CF02C127
:1008F0008D3409F461C08F3409F0BBCF13C0883543
:1009000009F4EEC0893538F4833509F49CC0863586
:1009100009F0AFCF76C0833709F4B8C08A3709F041
:10092000A8CF4EC180922701810118C0C201019752
:10093000F1F7939490DE882321F49AEF9916B1F79A
:1009400098CFE9EFE91508F494CF8EDEF801819392
:100950008F0189859A85E817F90711F09924EACF64
:100960006B814C812D818A8170E050E030E07EDD2A
:100970007DCF80922701810118C0C2010197F1F754
:10098000939469DE882321F49AEF9916B1F771CF19
:10099000E9EFE91508F46DCF67DEF80181938F0167
:1009A0008B859C85E817F90711F09924EACF6B81B4
:1009B0008A8170E071DD5ACF80922701810118C0D1
:1009C000C2010197F1F7939446DE882321F49AEF50
:1009D0009916B1F74ECFE9EFE91508F44ACF44DE96
:1009E000F80181938F018D859E85E817F90711F035
:1009F0009924EACF8A816B81605380534C81B1DDA9
:100A000035CF80922701810118C0C2010197F1F70B
:100A1000939421DE882321F49AEF9916B1F729CF18
:100A2000E9EFE91508F425CF1FDEF80181938F0166
:100A30008B859C85E817F90711F09924EACF8A8104
:100A40006B81C7DD13CF80922701810118C0C201DD
:100A50000197F1F79394FFDD882321F49AEF99161B
:100A6000B1F707CFE9EFE91508F403CFFDDDF80191
:100A700081938F018B859C85E817F90711F09924E4
:100A8000EACF8A8180536B8191DDF0CE809227017D
:100A900004C0C2010197F1F79394DDDD882321F4AE
:100AA00099EF9915B0F7E5CEE9EFE91508F4E1CE35
:100AB000DBDD8A83803311F486E603C0813321F4C1
:100AC00085E625DDC0DDD2CE823311F484E6F9CF90
:100AD000833311F481E6F5CF843309F0C7CE61C0CA
:100AE0008092270102C01092270139DDEADC5CDD2B
:100AF00082DDBCCE8092270104C0C2010197F1F7CC
:100B00009394A9DD882321F4F9EFF915B0F7B1CE5C
:100B100089EF891508F4ADCEA7DD8A83803359F4B7
:100B20000BE111E0F80181918F018DDDF1E00232DE
:100B30001F07C1F79BCE8133A1F48091220183DD91
:100B40008091230180DD809124017DDD0EE211E0A2
:100B5000F80181918F0177DDF1E002331F07C1F7C2
:100B600085CE823381F40AE211E0F80181918F0190
:100B70006ADDF1E00E321F07C1F78091320163DDBB
:100B8000809133019FCF833371F486E6C0DC5BDD57
:100B900085E6BDDC58DD84E6BADC55DD81E6B7DCF0
:100BA00052DD80E68ECF843309F060CE83E04BDDEA
:100BB00080E049DD82E047DD81E045DD88E682CFE7
:100BC00080922701862D3FDD0894611C711C8FEFF8
:100BD0006816710409F00CF449CE6624772446CED9
:100BE00080913F02823509F466C0833570F48C34FD
:100BF00051F18D3420F4873409F042CE61C08D3438
:100C000049F18F3409F03CCE11C0883509F453C046
:100C1000893530F4833571F1863509F031CE24C041
:100C2000833779F18A3709F02BCEB4C06091410245
:100C300040914202209143028091400270E050E0D6
:100C400030E014DCB3C0609141028091400270E05A
:100C500023DCACC08091400260914102605380531C
:100C6000409142027EDCA2C080914002609141022C
:100C7000B0DC9CC08091400280536091410296DCC0
:100C800095C080914002803311F486E610C0813314
:100C900011F485E60CC0823311F484E608C0833376
:100CA00011F481E604C0843309F080C080E62FDCB3
:100CB00080934A027BC053DC04DC76DC9CDC76C08B
:100CC00080914002803359F4EBE1F1E0AAE4B2E014
:100CD00081918D9391E0E232F907D1F767C08133BA
:100CE000B9F48091220180934A028091230180937C
:100CF0004B028091240180934C02EEE2F1E0ADE4DE
:100D0000B2E081918D9381E0E233F807D1F74EC0D4
:100D10008233C9F480912A0180934A0280912B0189
:100D200080934B0280912C0180934C0280912D0185
:100D300080934D028091320180934E028091330165
:100D400080934F0233C08333A9F486E6E0DB8093BF
:100D50004A0285E6DCDB80934B0284E6D8DB809395
:100D60004C0281E6D4DB80934D0280E6D0DB809399
:100D70004E021CC08433D1F493E090934A02109247
:100D80004B02E2E0E0934C0280924D02F8E6F093D1
:100D90004E020CC060924A020894611C711C8FEFD5
:100DA0006816710419F014F06624772480913F02CC
:100DB000823519F41092270102C080922701109207
:100DC0003F028091460280935102AA24BB24650110
:100DD00090E2E92E91EAF92E97E0092F112D50CDDE
:100DE000DA019330B1F0943028F4913041F0923030
:100DF00079F50AC0913211F1923251F524C0ECEC30
:100E0000F0E022E130E028C0EEEDF0E022E230E058
:100E100023C0813049F0813018F08230C9F40AC013
:100E2000E0E0F1E0849103C0E4E0F1E08491282F58
:100E300030E012C0E4E3F1E08491F9CFE0EFF0E0BC
:100E400029E030E009C0ECEAF0E020E230E004C044
:100E5000E0E0F0E020E030E0ED93FC93C90108957C
:100E60009C0140915F03509160034617570718F4A7
:100E7000F90190E045C06115710511F0AB01F8CFA3
:100E80008091E8008E778093E80040E050E0F0CF5A
:100E900080915803882309F445C0853009F444C083
:100EA0008091E80083FF02C081E008958091E8000E
:100EB00082FD32C08091E80080FF22C08091F30063
:100EC0009091F200782F60E0292F30E0262B372B0D
:100ED00007C081918093F100415050402F5F3F4FF8
:100EE0004115510519F02830310598F390E028306C
:100EF000310509F491E08091E8008E778093E80055
:100F00004115510529F6992319F606C08091580319
:100F1000882341F0853041F08091E80082FFF6CFD0
:100F200080E0089582E0089583E008959C016115B2
:100F3000710529F48091E8008B778093E800F9012E
:100F400027C080915803882399F1853099F18091C9
:100F5000E80083FF02C081E008958091E80082FFED
:100F6000F0CF06C08091F10081936150704059F03C
:100F70002091F3008091F200322F20E090E0822B4C
:100F8000932B892B79F78091E8008B778093E80089
:100F900061157105B1F606C080915803882341F0B0
:100FA000853041F08091E80080FFF6CF80E0089521
:100FB00082E0089583E008959C0140915F03509181
:100FC00060034617570718F4F90190E046C0611511
:100FD000710511F0AB01F8CF8091E8008E77809316
:100FE000E80040E050E0F0CF80915803882309F4F6
:100FF00047C0853009F446C08091E80083FF02C0F5
:1010000081E008958091E80082FD34C08091E8007D
:1010100080FF23C08091F3009091F200782F60E070
:10102000292F30E0262B372B08C084918093F100C4
:101030003196415050402F5F3F4F4115510519F0F7
:101040002830310590F390E02830310509F491E023
:101050008091E8008E778093E8004115510521F6D4
:10106000992309F0C1CF06C080915803882341F02D
:10107000853041F08091E80082FFF6CF80E008954E
:1010800082E0089583E00895BF92CF92DF92EF92BD
:10109000FF920F931F93CF93DF93182F092F7B019C
:1010A0006A01D9D0B82E8823B1F5812F902F9C01E9
:1010B000E901C114D10439F0F60180819181E81A67
:1010C000F90AC80FD91F00E010E022C08091E800A3
:1010D00085FD16C08091E8008E778093E8007ED36E
:1010E000C114D10449F0F60180819181800F911FD4
:1010F0009183808385E010C0AED0882349F00CC076
:1011000089918093F1000894E108F1080F5F1F4F67
:10111000E114F104D9F68B2DDF91CF911F910F913E
:10112000FF90EF90DF90CF90BF900895382F282F39
:101130002EC0822F8F708093E900231721F4762F21
:10114000942F50E006C07091EC009091ED0050910A
:10115000F00091FF1BC08091EB008E7F8093EB002D
:101160008091ED008D7F8093ED008091EB00816098
:101170008093EB007093EC009093ED005093F0009F
:101180008091EE0087FD02C080E008952F5F273038
:1011900080F23F703093E90081E008950F931F9330
:1011A000CF93DF93062FEC0110E02AC0988199239A
:1011B00029F16B81E981FA812C81892F8F70873029
:1011C00018F5223010F452E001C056E040E028E06B
:1011D00030E003C04F5F220F331F2E173F07D0F3BD
:1011E0006295660F660F607C991F9927991F692B7E
:1011F0004295407F452B9ADF882331F01F5F25966B
:101200001017A0F281E001C080E0DF91CF911F9123
:101210000F9108958091590388239CF404C0809114
:1012200058038823B9F08091E80082FFF8CF8091BD
:10123000E8008B778093E800089580915803882315
:1012400049F08091E80080FFF8CF8091E8008E7728
:101250008093E80008954091E4005091E50024E671
:101260008091EC0080FF24C08091E80080FD1EC0CA
:1012700080915803882311F482E00895853011F499
:1012800083E008958091EB0085FF02C081E008951E
:101290008091E4009091E5008417950709F32223DB
:1012A00011F484E008952150AC01DACF80E0089574
:1012B0008091E80082FFDCCFF9CFEF92FF920F938D
:1012C0001F934FD056D008ED10E0F80180818F7742
:1012D000808380818068808380818F7D808319BC3A
:1012E0001092580310925403109256031092550313
:1012F00080EEE82EF12CF70180818B7F8083F8014E
:1013000080818160808380E060E042E00FDFE1EE79
:10131000F0E080818E7F8083E2EEF0E0808181606A
:101320008083808188608083F70180818E7F8083C5
:10133000F8018081806180831F910F91FF90EF9071
:101340000895E8EDF0E080818F7E8083E7EDF0E0A6
:1013500080818160808384E082BF81E08093570335
:10136000ACCFE8EDF0E080818E7F80831092E200C8
:1013700008951092DA001092E10008951F920F92E2
:101380000FB60F9211242F933F934F935F936F9358
:101390007F938F939F93AF93BF93EF93FF9380912E
:1013A000E10082FF0AC08091E20082FF06C08091C6
:1013B000E1008B7F8093E100A5D98091DA0080FF66
:1013C0001DC08091D80080FF19C08091DA008E7F07
:1013D0008093DA008091D90080FF0CC080E189BD44
:1013E00082E189BD09B400FEFDCF81E080935803FE
:1013F00082D904C019BC109258037ED98091E100B3
:1014000080FF18C08091E20080FF14C08091E2004C
:101410008E7F8093E2008091E20080618093E20001
:101420008091D80080628093D80019BC85E08093B9
:101430005803D3D18091E10084FF2FC08091E20056
:1014400084FF2BC080E189BD82E189BD09B400FE23
:10145000FDCF8091D8008F7D8093D8008091E100EE
:101460008F7E8093E1008091E2008F7E8093E20086
:101470008091E20081608093E20080915403882390
:1014800011F084E007C08091E30087FD02C081E095
:1014900001C083E080935803A0D18091E10083FFD5
:1014A00022C08091E20083FF1EC08091E100877F0F
:1014B0008093E10082E0809358031092540380915E
:1014C000E1008E7F8093E1008091E2008E7F809327
:1014D000E2008091E20080618093E20080E060E0C1
:1014E00042E024DE7AD1FF91EF91BF91AF919F91BD
:1014F0008F917F916F915F914F913F912F910F90BD
:101500000FBE0F901F9018951F93DF93CF93CDB709
:10151000DEB7AC970FB6F894DEBF0FBECDBFE9E5DE
:10152000F3E08091F100819323E0E136F207C9F7FF
:101530002DD98091E80083FF38C180915903309103
:101540005A03353009F487C0363040F43130C9F1E0
:10155000313070F0333009F028C133C0383009F42D
:10156000F5C0393009F404C1363009F01EC196C007
:10157000803821F0823809F018C108C090915503D5
:1015800080915603882399F0926011C080915D0389
:101590008F708093E9008091EB0090E025E09695B4
:1015A00087952A95E1F7982F91701092E900809124
:1015B000E800877F8093E8009093F1001092F1009B
:1015C000D0C0882319F0823009F0EFC090E08F710D
:1015D0009070009721F0029709F0E7C00CC080914D
:1015E0005B03813009F0E1C010925603333069F596
:1015F000809356032AC080915B03882331F52091A4
:101600005D032F7009F4D1C02093E9008091EB00B5
:1016100080FF1BC0333021F48091EB00806213C047
:101620008091EB0080618093EB0081E090E002C04C
:10163000880F991F2A95E2F78093EA001092EA003A
:101640008091EB0088608093EB001092E90080911C
:10165000E800877F89C0882309F0A7C010915B0349
:101660001F778091E3008078812B8093E300809145
:10167000E800877F8093E800CDDD8091E80080FF5F
:10168000FCCF8091E30080688093E300112311F484
:1016900082E001C083E08093580387C08058823085
:1016A00008F083C080915B0390915C0323E08C3D44
:1016B000920709F033C083E08C838AE28B837FB783
:1016C000F894DE0115966EE040E050E011E2E62F5E
:1016D000F0E010935700849140FF03C082958F7013
:1016E0006F5F8F70282F30E08A3018F0C901C796DD
:1016F00002C0C901C0968D939D934F5F5F4F4431E7
:10170000510529F77FBF8091E800877F8093E8002B
:10171000CE0103966AE270E0A3DB12C060915D0324
:10172000AE014F5F5F4F5CDBBC01009709F43DC029
:101730008091E800877F8093E80089819A813CDC72
:101740008091E8008B778093E8002FC0803869F59E
:101750008091E800877F8093E80080915403809314
:10176000F1008091E8008E778093E80053DD1DC082
:101770008823D9F490915B039230B8F48091E8000B
:10178000877F8093E8009093540344DD8091540355
:10179000882331F48091E30087FD02C081E001C01D
:1017A00084E0809358030E94CA038091E80083FF7D
:1017B0000AC08091E800877F8093E8008091EB0069
:1017C00080628093EB00AC960FB6F894DEBF0FBE3C
:1017D000CDBFCF91DF911F91089508951F93809100
:1017E0005803882371F01091E9008091EC00109269
:1017F000E9008091E80083FF01C086DE1F7010932E
:10180000E9001F9108954F925F926F927F928F929D
:101810009F92AF92BF92CF92DF92EF92FF920F937F
:101820001F93DF93CF9300D00F92CDB7DEB77C012B
:101830006DB67EB680915803843009F09AC020912D
:10184000E4003091E500F7018285938582179307C4
:1018500009F48FC081818F708093E9008091E80046
:1018600085FF87C05DB64EB6408550E08DB79EB708
:10187000841B950B0FB6F8949EBF0FBE8DBF0DB79E
:101880001EB70F5F1F4F19821B821A82C02E912E26
:10189000C80160E070E050E001D2C701BE016F5F97
:1018A0007F4F40E098018E010E5F1F4F0E94A603FC
:1018B000882EF70184859585892B19F4AA24BB24E9
:1018C0000BC020E0F70186859785892B09F021E080
:1018D00081E02827A22EBB24F7010681178101157C
:1018E000110511F4DD2412C04A815B818C2D992DE4
:1018F000B801BED1DD24009711F0DD24D394F701A7
:101900004085C8016C2D792D50E0BFD18A819B8123
:10191000892B01F1882021F4DD2011F4AB28D1F0CE
:10192000F701848595859787868781818F7080935D
:10193000E9008981882311F08093F1006A817B811D
:101940008C2D992D40E050E09FDB8091E8008E7750
:101950008093E8008091E4009091E500F70193877F
:101960008287252D342DC9010FB6F8949EBF0FBE76
:101970008DBF0FB6F8947EBE0FBE6DBE0F900F9058
:101980000F90CF91DF911F910F91FF90EF90DF901B
:10199000CF90BF90AF909F908F907F906F905F900F
:1019A0004F900895CF93DF93DC010996FC0187E007
:1019B000EF0119928A95E9F781E019968C931997AE
:1019C00084EF91E01D969C938E931C9783E0149670
:1019D0008C931497CD01019661E0E0DB811181E0E9
:1019E000DF91CF9108956F927F928F929F92AF92E5
:1019F000BF92CF92DF92EF92FF920F931F93DF93EC
:101A0000CF9300D00F92CDB7DEB76C016DB67EB626
:101A10008091E80083FF15C1F601808190E020915C
:101A20005D0330915E032817390709F00AC18091E0
:101A30005A03833009F4ADC0843030F4813071F042
:101A4000823009F0FEC0E1C08A3009F4C6C08B3094
:101A500009F4B0C0893009F0F4C057C0809159032F
:101A6000813A09F0EEC09DB68EB61B821A82809133
:101A70005B0310915C038983F601408550E08DB7CC
:101A80009EB7841B950B0FB6F8949EBF0FBE8DBFFB
:101A9000EDB6FEB60894E11CF11CBE2CAF2CC701BC
:101AA00060E070E050E0FAD01150C601BE016F5FF7
:101AB0007F4F412F97018E010E5F1F4F0E94A6039B
:101AC000F601268137812115310529F04085C901AC
:101AD000B70150E0DAD01092E9008091E800877FEA
:101AE0008093E8006A817B818B2D9A2DB9D98091F2
:101AF000E8008B778093E800292D382DC9010FB6B7
:101B0000F8949EBF0FBE8DBF9CC080915903813257
:101B100009F097C09DB68EB600915F0310916003E7
:101B2000A0905B03B0905C038DB79EB7801B910BB8
:101B30000FB6F8949EBF0FBE8DBFEDB6FEB60894EB
:101B4000E11CF11C8091E800877F8093E800C701C9
:101B5000B801ECD98091E8008E778093E80080E0AE
:101B600090E0AA2011F081E090E0BA94E80EF91E0E
:101B7000081B190BC6016A2D4B2D97010E948E037D
:101B8000892D982D9C010FB6F8943EBF0FBE2DBF36
:101B900058C080915903813A09F053C08091E80000
:101BA000877F8093E8008091E80080FFFCCFF601FA
:101BB00081853FC080915903813209F042C08091F4
:101BC000E800877F8093E80025DB90E080915B034D
:101BD000811191E0F601918734C0809159038132DF
:101BE00081F58091E800877F8093E80013DB809186
:101BF0005B0390915C03807036E0969587953A95EB
:101C0000E1F7F601958784871CC080915903813ADA
:101C1000C1F48091E800877F8093E8008091E8001C
:101C200080FFFCCFF60184859585969587959695DE
:101C300087958093F1008091E8008E778093E8008B
:101C4000E9DA0FB6F8947EBE0FBE6DBE0F900F900E
:101C50000F90CF91DF911F910F91FF90EF90DF9048
:101C6000CF90BF90AF909F908F907F906F9008958E
:101C7000FB01DC0104C08D910190801921F44150D9
:101C80005040C8F7881B990B0895FB01DC0102C086
:101C900001900D9241505040D8F70895DC0101C0E9
:0E1CA0006D9341505040E0F70895F894FFCF47
:101CAE00008108000001340108000000000000005F
:00000001FF
